:030000000219FDE5
:03000B000200AA46
:03002B0002019C33
:03005B0002034F4E
:0300730002033550
:1000800002030406080C10182030406080040608A3
:100090000C10182030406080A0C000070F1F3F0DDB
:1000A0000D04050D050305030302C2AF306308C24A
:1000B00063857C8AD2AF32C0D0C0E0206227E525BC
:1000C0006002E473E525F4C3334009758A00D26306
:1000D000F57C01D6F58A758B00758D00D262D0E073
:1000E000D0D0D2AF32C3E526334009758A00D2633F
:1000F000F57C01F6F58AC262E526F4603C306803BF
:10010000207213758B00758D00D0E0D0D0C295C2DF
:1001100094C293D2AF32C295C294C293206E0D2086
:10012000660A7414D5E0FDE57EF45290758B007577
:100130008D00D0E0D0D0D2AF32758A00D263757C0A
:1001400000C28DD262212C01C4306805206602D223
:100150009501C4306805206602D29401C430680558
:10016000206602D29301C4D29230680A20660774D6
:1001700010D5E0FDD29501C4D29130680A206607FF
:100180007410D5E0FDD29401C4D290D29230680AA6
:100190002066077410D5E0FDD29301C4C2AFC2AD92
:1001A00053E6EFC0D0C0E0D2D3D2AFE57D6009E521
:1001B0007A6005757A0041E2757A01C2CEE52A605F
:1001C00007207449152A410D7800790020742EE526
:1001D00080307E01F430E70278FF53DACF207E03CF
:1001E00043DA20307E0343DA10C2D8C271E5803092
:1001F0007E01F430E70279FFC3E89970CB306103E8
:10020000752A18207403752A18885FD27020740D1F
:10021000E52B6004152B411D43DA01C2D820700282
:10022000417BA85F206102C2702074367982B704D6
:1002300031C3E894F0400374F0F8E8C4540F28F890
:100240007984B703024162C313C3138721200802D4
:10025000C313200A06C3C898F8416228F8500374F3
:10026000FFF88822E52D54066011E533C313C3134C
:1002700024062522F52250037522FF7882B6045900
:10028000852224A824C3E52495644002A864C3E819
:1002900095664002A8668825E569700241CCC3E8EE
:1002A000AA699A5003E8FAE4F9EAC333FBE56BF470
:1002B0005B29400D256AF8E56A6002156A400B412A
:1002C000CC0AC3E56A9A5002056A78FF8826C26E96
:1002D000C3E52694F84002D26EC3E525944040025F
:1002E000D26420CF0AD0E0D0D043E610D2AD32C2E3
:1002F000CF053AE57D6009E57B6005757B00612BE4
:10030000757B017801E52A6005307402152AC3E582
:100310005F94014005756200612B756300756C0088
:10032000E5622401F56250037562FFD0E0D0D0434E
:10033000E610D2AD32C2AFC0D053E67FC260759135
:1003400000855694855795759104D0D0D2AF32C2AE
:10035000AF53E6EFC2ADC0D0C0E0C0F0D2D3D2AF51
:10036000A8FBA9FCE57D6007C3E913F9E813F8C20F
:10037000D830710261C153DACF207E0343DA1030E6
:100380007E0343DA20D271E580307E01F420E7025B
:10039000619888278928A1E853DACF207E0343DAC1
:1003A00020307E0343DA10C2D8C271307402A1D467
:1003B0007800E580307E01F430E702A1D4885FA1A7
:1003C000BC53DACF207E0343DA20307E0343DA10B9
:1003D000C271206102819A53DACF207E0343DA1082
:1003E000307E0343DA20C2D8D271885A895BC3E8D1
:1003F0009558F8E99559F97B007E087A00C3E8948E
:100400008CE994005005755E00818C882178A2E605
:10041000A8216055C3E894C8E994005008E4D2E4E8
:10042000FB7A0A8167C3E89468E994015008E4D232
:10043000E3FB7A0F8167C3E894D0E994025008E4A3
:10044000D2E2FB7A1E8167C3E894A0E994055008C4
:10045000E4D2E1FB7A3C8167C3E89498E9940850C0
:1004600008E4D2E0FB7A787E00C3E8955CFCE9956D
:0F0470005DFD30E70AECF42401FCEDF43400FDEF
:10047F00755E00C3EC9AED9E5003755E01885C8932
:10048F005D855A58855B597802A1BCC3E89527F85A
:10049F00E99528F9307C02A1A0307B02A1A0307A27
:1004AF0002A19920750281BDE9FDE8FC81DCE9C359
:1004BF0013F9E813F8307902A199E9C313F9E81396
:1004CF00F8307802A199E9C313FDE813FC206126E7
:1004DF00C3EC941CED9402400281F3ED7018C3EC51
:1004EF0094C850120529C3E529940A5002A1D47566
:1004FF005F00D270A1D4E529600215297888E6F94A
:10050F007400207F087896B90302789EE624FAFEDD
:10051F00E43400FFC3EC9EFCED9FFD9208B903107D
:10052F00A2085007207609D276A13F307602C27614
:10053F00A2085016B9030DECF42401FCEDF43400BD
:10054F00FD02055978007900A1A0B90315EC33FC21
:10055F00ED33FDC3EC940AFCED9400FD50047C00D8
:10056F007D00C3EC94FFED9400400678FF7900A165
:10057F00A0EC8575F0A4C5F0A2F733F8790040031D
:10058F000205BC78FF79000205BCE9C313F9E81333
:10059F00F8307C0EE9600278FFC3E81338F8E434D2
:1005AF0000F9C3E894FFE99400400278FF885FD216
:1005BF0070206102A1D4741FF4552F4BF52FC27414
:1005CF00EB7002D274752A18307403752A0A3061E1
:1005DF0002A1E820740353DAFE207403752B06D0B2
:1005EF00F0D0E0D0D0D2AD43E61032790102061838
:1005FF007903020618790A020618791E020618797D
:10060F006402061879C80206187817E4D5E0FDD8F9
:10061F00FAD9F6227A147B7802063F7A107B8C0285
:10062F00063F7A0D7BB402063F7A0B7BC802063F6A
:10063F007902B27DE4D291D5E0FDD294D5E0FDC22E
:10064F0094D5E0FDC291D5E0FDD295E576D5E0FDDC
:10065F00C2957496D5E0FDD9D9EAF8D5E0FDD8FB5F
:10066F00DBCED29122C37C007D0075F00005F0EA4D
:10067F0033FAEB33FB50F6EB13FBEA13FAC3E9FF44
:10068F00E8FEE89AF8E99BF95004EFF9EEF8B3ECBD
:10069F0033FCED33FDD5F0DFEDF9ECF822E889F00E
:1006AF008A20D2D4F8A9F07B0030F70B7BFFF4241B
:1006BF0001F8E9F43400F9E88520F0A4ADF0F8E989
:1006CF008520F0A4AFF0FEED2EF974003FFA7C0404
:1006DF00C3EA13FAE913F9E813F8DCF48BF030F7F7
:1006EF000AE8F42401F8E9F43400F9E889F0C2D4F7
:1006FF00F8A9F0227882B6040302075EC3E55F947F
:10070F00014003020728852224E4F545F546F54705
:10071F00F548F549C26D02075E7882E6FCD26DE5B9
:10072F0022F523783879C7AA40AB41C3EB13FBEA14
:10073F0013FAEC146013C3EB13FBEA13FAEC141463
:10074F006007C3EB13FBEA13FAD17488458946227D
:10075F00C3E5459523F8E5469400F9500CC3E8949A
:10076F0080E994FF401602078FC3E8947FE9940055
:10077F00500302078F787F790002078F788079FF07
:10078F00884A894B22E54A2547F8E54B3548F985D4
:10079F004B20E4300701F43549FA30E709C3EA94F6
:1007AF00F040150207CDC3EA940F50030207CD782E
:1007BF00FF79FF7A0F0207CD780079007AF0C3E551
:1007CF00249564500AC374019524500B0207EBE57E
:1007DF004B20E70E0207EBE54B30E70688478948C9
:1007EF008A492278A4E6FAC3E54A33F8E54B33F990
:1007FF001206ACE930E70BC3E89480E994FF40138D
:10080F000126C3E8947FE9940050020126787F798E
:10081F00000126788079FFE820E715C3E52398F8D3
:10082F004009C3E89401400302084D780102084DC6
:10083F00E8F424012523F8400302084D78FF884C83
:10084F002278A5E6FAA848A9491206ACE930E70CC8
:10085F00C3E89401E994FF4016020882C3E894FFAD
:0F086F00E99400500302088278FF7900020882A2
:10087E00780179FFE920E715C3E54C98F84009C3E4
:10088E00E8940140030208A978010208A9E8F424BB
:10089E0001254CF840030208A978FF88242278FF2E
:1008AE00C26420693D206A12D264C3E541940A40B5
:1008BE0009C3E52594405002C26479A1E76023E59F
:1008CE0041601F74FF8541F0848539F0306A0375ED
:1008DE00F005A4F8C5F0600278FFC3E895675002F2
:1008EE00A867886622C3E54094C8E5419400E56692
:1008FE005003142104046002F5662202090C2275CD
:10090E00E890227883E6FFE5E820ECF7A8BDA9BEC3
:10091E000573C3E57394084052757300E9FA79A024
:10092E00E76044EA7007E574601B020947C3E89567
:10093E00746010E5745006600C140209530460F9DB
:10094E00020953E574F574C39472401B7564C0C3F9
:10095E0094044013756480C39404400B756440C3C3
:10096E009404400375640075BB0622E564241050A0
:10097E000274FFF5647982B7040221A0C3A864E56E
:10098E0024985002A824C3E895664002A8668825DC
:10099E008826E573B4070375BB1022743279A687D7
:1009AE00F0A4C5F0A2F733F8C3E895644002A8643A
:1009BE0088228824882588268867227540007541FC
:1009CE00F022C2AF75C820A8CCA9CDAA3A30CF016B
:1009DE000A75C824D2AFC3EA13FAE913F9E813F87B
:1009EE00AB3BAC3C883B893CC3E89BF8E99C206957
:1009FE000A547FF930670241F34150AD3D8A3DF90B
:100A0E00EA9D547FFA600478FF79FFAE3EAF3F8BCC
:100A1E003E8C3FC3EC9FFCC3E99CF542A83BA93C2E
:100A2E00C3E89EF8E99FF9C3E54113FBE54013FACD
:100A3E00E82AF540E93BF54150067540FF7541FF48
:100A4E00419AAA40AB41AC40AD417E047F02C3EB5C
:100A5E00940440021E1FC3EB940840021E1FC3EDF8
:100A6E0013FDEC13FCDEF7C3EA9CFAEB9DFBEF6083
:100A7E0009C3E913F9E813F8DFF7EA28FAEB39FBB3
:100A8E008A408B4150067BFF8B408B41C3EB940217
:100A9E005002D2673069047F0341C57892E6FFC3E6
:100AAE00E537948240110FC3E53794A040010FC380
:100ABE00EF940640027F057E03E541C4540FF9E52D
:100ACE0041C454F0F8E540C4540F28F8C3E89EFA28
:100ADE00E99400FB4009C3EA9402EB940050047AB7
:100AEE0002E4FB613FAA40AB41EBC4FEEAC4540FE3
:100AFE004EFCC3EA9CFAEB9400FBC3E813C313F855
:100B0E00EA28FAEB3400FB8A408B41C3EB94024097
:100B1E0002C2677803EBC4FE7B00EAC4540F4EFAA0
:100B2E00C3EA98FA4005C3940250027A027892E61C
:100B3E00FF306002613F855256855357D26043E6BF
:100B4E0080C3E49AF8E49BF9C3E833F8E933F9304B
:100B5E00670261E0E8FAE9FBD3E913FDE813FC88CC
:100B6E00528953C3EF94036038EF20E00DE82CF860
:100B7E00E93DF9ECFAEDFB020B9BE828F8E939F9AF
:100B8E00C3E82402F8E93400F97AFE7BFFC3EF9440
:100B9E0003400E8A548B55884E894F8C508D51814F
:100BAE0014885489558A4E8B4F8C508D5130692044
:100BBE00C3E53394034019E542A2E713F8E555F473
:100BCE00240138400B20E7087554FFF42401F55535
:100BDE008114E8FAD3E813FC8852C3EF9403602023
:100BEE00EF20E007E82CF8ECFA8100E8282402F860
:100BFE007AFEC3EF940340088A54884E8C508114B9
:100C0E0088548A4E8C50E56BC3335002646BF56B7F
:100C1E00306002811E753404D26043E680E52D54A7
:100C2E0006601FA840A941C2AF53E67F759100C36D
:100C3E00E498F594E499F595759104D26043E680B5
:100C4E00D2AF22D265754400752000306B0375203B
:100C5E0040020C70D265754400752040306B0375F0
:0F0C6E002000D2AF7801206722E52D54066002E6
:100C7D00C265C3E541940540137802940540087898
:100C8D0003940540027806306902780A206019E560
:100C9D0044601530690AC3E53394034003D5340627
:100CAD00D2AFD26CA1529126D2AF0000C2AF206755
:100CBD002AE541C3FB940F40027B0FEB24053073F3
:100CCD000123306A02742820620123F93069027908
:100CDD0082E58D13E58B13C39940B10544E59B5413
:100CED0040B52002A13C30690A08C3E8940A4001CE
:100CFD000881992065028170C26553E67F75910068
:100D0D003067107594007595FC759104D26043E6BB
:100D1D00808170AE40AF41C3EE33FEEF33FF500420
:100D2D007EFF7FFFC3E49EF594E49FF595A116C366
:100D3D00E5339402500281703065028170D802A1B2
:100D4D00508199C26C53E67F7591008554948555F9
:100D5D0095759104854E56854F57D26043E680D2E6
:100D6D00AFE52D54066008206A020533020D8C3064
:100D7D006C0D206B0A2065071581158102160D2259
:100D8D0078003064053065027801E53775F007A409
:100D9D00F9E5F028F5F0E9A2F013A2F113A2F21390
:100DAD00F537C394785003753778C3E537953840D8
:100DBD0008D266C295C294C293306002A1C6855016
:100DCD0056855157D26043E68022207D11C2AF7502
:100DDD004302D291C292D2AF759F11020FAEC2AF34
:100DED00754302D291C290D2AF759F11020FAE30F2
:100DFD007245207D22C2AF754303900178757E0246
:100E0D00C293D290D292306204D294C11CC291D2BC
:100E1D00AF759F01020FAEC2AF7543039001787598
:100E2D007E02C295D292306204D294C13CC291D25C
:100E3D00AF759F21020FAE207D17C2AF7543039092
:100E4D000153C293306202D294D2AF759F01020F4B
:100E5D00AEC2AF754303900153C295306202D29476
:100E6D00D2AF759F21020FAE207D11C2AF75430425
:100E7D00D292C290D2AF759F21020FAEC2AF754311
:100E8D0004D290D292C292D2AF759F01020FAE30B2
:100E9D007243207D20C2AF754305900167757E04B6
:100EAD00C294D291306204D295C1BAC292D2AF75BA
:100EBD009F11020FAEC2AF754305900189757E017A
:100ECD00C294D291306204D293C1DAC290D2AF757E
:100EDD009F11020FAE207D17C2AF754305900149DA
:100EED00C294306202D295D2AF759F11020FAEC27D
:100EFD00AF75430590015DC2943062EBD293D2AFD2
:100F0D00759F11020FAE207D13C2AF754306D290AF
:100F1D00D292C291D2AF759F01020FAEC2AF75438F
:100F2D0006D292C291D2AF759F21020FAE3072449C
:100F3D00207D20C2AF754301900189757E01C29558
:100F4D00D292306204D293E158C290D2AF759F21F4
:100F5D00020FAEC2AF754301900167757E04C29357
:100F6D00D290D292306204D295E17AC292D2AF750C
:100F7D009F01E1AE207D16C2AF75430190015DC2A8
:100F8D0095306202D293D2AF759F21E1AEC2AF759B
:100F9D004301900149C293306202D295D2AF759F41
:100FAD0001C26622900147757E00C295C294C2931C
:100FBD00D292D291D290C2622278807609087609B7
:100FCD000876040876FF0876030876FF08760A0887
:100FDD007603087601087601788C76010876FF088D
:100FED0076FF0876FF0876FF0876FF087603087609
:100FFD00FF0876FF0876FF0876250876D008762854
:10100D000876500876040876FF0876020876000800
:10101D00767A0876FF08760108760108760008765C
:10102D0003227887E6FFC272BF0302D2727888E688
:10103D00C394036008C27DE630E102D27DC27E78A2
:10104D0089E630E102D27EC3EF94026008758E010D
:10105D00D273021067758E00C273227880E61490E9
:0E106D0000809378A4F67881E61490008093BA
:10107B0078A5F67886E61490008D9378A6F6789C82
:10108B00E67538FF75390CB402067538A075390A48
:10109B00B4030675388275390578A3E61490009A67
:1010AB0093F569120FB122227896E6FA7897E6FB50
:1010BB007888E6B40305C3EB940EFB307F047A000B
:1010CB007BFFC3EB9AFCC3948250027C8275750044
:1010DB000575EC8575F0A4C3E5F0947D40F222D242
:1010EB007F11B31206097A007B007C101205FFE515
:1010FB005F2AFA74003BFBDCF37C04C3EB13FBEAC3
:10110B0013FADCF7FEC27F11B322E5EF20E603757D
:10111B0020000520903FFFE520146006901FFF1470
:10112B0060009304600375EF1253D9BF7581C04300
:10113B00FF801205FA75EF0243B203E5B3240420D6
:10114B00E70DF521E5E320E0068521B343E301122A
:10115B000FB17580FF75A40075F19075D47F7590F4
:10116B008775A5BF75F2BF75D50075A60175E241F0
:10117B00E4F8F6D8FD756B01120FC6121657789866
:10118B008676753001C2AF120613120623120609BA
:10119B0012062A120609120631120609C2AF78FA94
:1011AB0079FA308707D9FBD8F7021C00112F116889
:1011BB0011B211B378988676120FB175B68075A9F6
:1011CB0000757D0075885075891275C8247591045A
:1011DB0075D84075A82275B80275E690759B807519
:1011EB009D0075D10E75BC5875BB0675BA1175E8A7
:1011FB00801205FAD2AF12090953DACF207E0343CE
:10120B00DA20307E0343DA1043DA01C2D8C27112FE
:10121B000613D2617B037A0CE55E70077A0CDB0355
:10122B000211A71206092070030211A7C270E55F15
:10123B00C3940240E1E52F541F856160F561B560F1
:10124B00D5DAD5C26153DACF207E0343DA20307E64
:10125B000343DA10C2D8C27178A2E67008D274E5E3
:10126B002F54E0F52FC27575290012060E30740944
:10127B00C3E529940A4002D2751205FF7802307437
:10128B00027800C3E55F9840F0C2AF120623120646
:10129B0023120623D2AF120613754D007888E6B4DD
:1012AB00030261851205FF788CE6C394015003029B
:1012BB001385E530C394015003021385207435C3A5
:1012CB00E55F94FF5003021385C2AF120638D2AF0D
:1012DB0012060EC3E55F940150EFC2AF1206231244
:1012EB000604120623D2AF12060EC3E55F94FF402D
:1012FB00E90217FF7F02D27F11B312060EC2AFC2F3
:10130B007F11B3AE5FC3E55F947FD2AF407612051A
:10131B00FAC2AF120638D2AFDFDC11EAC3EE940586
:10132B007897F61206131216991217827F0AD27F3C
:10133B0011B312060EC2AFC27F11B3AE5FC3E55F2E
:10134B00947FD2AF50E61205FAC2AF1206231206F3
:10135B0004120623D2AFDFD611EAEE24057896F6F7
:10136B001206131216991217B112060E11B3C3E51A
:10137B005F94FF500241C70217FFC3E55F954D40D5
:10138B0003855F4D12060E78017988E7B403027866
:10139B0005C3E55F98400241A7C2AF12063812069B
:1013AB0038120638D2AF120613753000E4F531F55A
:1013BB00320531E531F470390532789AE678191433
:1013CB006012783214600D787D14600878FA14601E
:1013DB0003753200C3E53298401715327531B47876
:1013EB00998676C2AF120638D2AF789886761206F7
:1013FB000E120604E52A700530740221A77801202D
:10140B0074027806C3E55F9840A77888E6C3940317
:10141B00600312060EE52A70030211A7C2AF120F6A
:10142B00B1E4F522F523F524F525F526F56AD2AFBF
:10143B007885E6C333F568E4F545F546F547F54899
:10144B00F549F573F52CF52DF53775730875BB104C
:10145B001205FA12090DE5E820ECFBA8BDA9BEE9BF
:0E146B007001F8887412091175730875BB10B2
:101479007887E6FE7602112F7887EEF6C2AF75649B
:10148900FF1209A9852264852265852266D2AF7576
:10149900220175240175250175260185636C756D19
:1014A9000175B69075A903757D017888E6B40307BF
:1014B900C27D307602D27DD268D269753300120FAF
:1014C90013120F3A1209C91209D01209C91209D007
:1014D9001209C90214EBC2AF112FD2AF757300758F
:1014E900BB06120C62120703120D8D120DD71209D9
:1014F900D0120C51306D0312075F2067031208AC3C
:101509003067031208F3120D8D120DFC1209D01267
:101519000C62306D03120794120D8D120E751209AB
:10152900D0120C51306D031207F2120D8D120E9C60
:101539001209D0120C62306D03120850120D8D126F
:101549000F131209D012090D120C51120D8D120F21
:101559003A1209111209D0306935206B3285676456
:1015690085676585636C756D0179187A0CC3E533F8
:1015790099400FC269D26A8A3585676485676602B0
:101589001598C3E55F940140030214EB0216153068
:101599006A1B206B18E535147004C26A81DFF535C2
:1015A900C3E55F940140030214EB0216157536007A
:1015B900C3E56278FA985054307404E52A604D788E
:1015C90088E6B40317207D05207607A1E530760269
:1015D900A1E5206B07D26B856764A12A78F0306B8F
:1015E900058567647820C3E54198500281EB306B2B
:1015F9001BC26BC27D307602D27DD26A75351285E7
:10160900676481EB0536E55F6002C118753600C273
:10161900AF120FB17887E6FE7602112F7887EEF6C2
:10162900E4F522F523F524F525F526F568C2687554
:10163900B68075A900757D00D2AF1205FA120FB1F7
:10164900307409C3E5369405400221A761B7901AA1
:101659000D78201216DBE520B4550CA31216DBE534
:1016690020B4AA03021679120FC612169902169807
:10167900901A0378807B0A1216DBA308DBF9901A0B
:101689000F788C7B181216DBA308DBF9901A272236
:10169900C2AF12171A1216F4901A00740E1216E03D
:1016A900A374041216E0A374141216E0901A0378B6
:1016B900807B0A1216DFA308DBF9901A0F788C7B5E
:1016C900181216DFA308DBF912172D12170B901A3F
:1016D9002722E493F622E6438F01538FFD75EF022B
:1016E90075B7A575B7F1F0538FFE22438F02438F6B
:1016F9000175EF0275B7A575B7F1901A0DF0538F03
:10170900FC22901A0D7455D1E0901A0E74AAD1E0FA
:10171900227A3079D07820901A40D1DBE520F70978
:10172900A3DAF7227A3079D0901A40E7D1E009A3F9
:10173900DAF922AB77A878BB01027980BB0202797A
:1017490081BB03027982BB04027984BB05027986D5
:10175900BB06027992BB07027987BB080279A3BB52
:101769000902799CBB0A027988BB0B027989E8F7DF
:10177900227C05120613DCFB22C2AF1206231206D5
:101789002A12063112063812060412062312062AF4
:1017990012063112063812060412062312062A12FC
:1017A9000631120638D2AF22C2AF120638120631FC
:1017B90012062A12062312060412063812063112DC
:1017C900062A1206231206041206381206311206D8
:1017D9002A120623D2AF22AE77AF78C2AF12062300
:1017E900120623120623120604DEF2120638120626
:1017F90004DFF8D2AF2212178212177A12177A75FC
:1018090077017578017579001217E07C05AD5F12D3
:101819000613C3ED955F70F5C3E55F9401400AC3F4
:10182900E55F94FF403702184312173C12169912CC
:101839001782C2AF75EF1212177ADCD10579C3E5A9
:10184900799403500280C112177A0578E5771490CC
:10185900009F93F808C3E57898500280A812177A78
:0E18690012177A0577C3E577940C500280942D
:0E187700120FC6121699C2AF75EF1212177A31
:0319FD00021115BF
:101A00000E0414090904FF03FF0A03010155AA018A
:101A1000FFFFFFFFFF03FFFFFF25D0285004FF0259
:081A2000007AFF01010003FF41
:101A4000234F76736B794D5232304150726F2320A1
:101A500023424C48454C492346333930232020202B
:101A60002020202020202020202020202020202076
:101C0000C2AFC2D353D9BF7581C043B20343FF8073
:101C1000752438752503B1C975EF0275E24043F1AB
:101C20008053A47F75D400D2877DFA780379E67C4F
:101C300010752200752300901DD67B0675249875BB
:101C400025013087028142208708D8FBD9F9DCF7CB
:101C500081B4308708D8FBD9F9DCF781B4B189E4C5
:101C600093A3C39A6004DDC381B4DBDBB17B600264
:101C7000812B7B08E493FAA3B15CDBF87A30B15C8A
:101C8000752200752300B17BEAFCEBFDC3ED94FEE9
:101C9000400EB17B8A278B28ED30E0048A828B834B
:101CA000B17B7AC270D8C3ED94FE601350CEBD00F4
:101CB00025EC60097520007521FF0200008100A855
:101CC00027A9280809D804D90281D3B17FEA89AAB3
:101CD000F281C50D81A0C3ED94035049EDA2E092BD
:101CE000007AC5C3E5829400E583941C50902000DF
:101CF00010438F02438F0175B7A575B7F1F030001F
:101D00001FA827A9280809438F01538FFDD804D99C
:101D100002A12089AAE275B7A575B7F1F0A3A10DBC
:101D2000538FFC817C7AC1BD030CE493A3FAB140CC
:101D3000DCF8B138817C817EAA22AB23B15CEBFA5E
:101D4000EA6222752608C3E52313F523E52213F57D
:101D50002250066323A0632201D526EAB1C9B1C986
:101D600075260AEAF4200102D287300102C287B147
:101D7000C9C3134002C201D526EB22B17FEAFB2082
:101D80008702A17F308702A184752608AE24AF2583
:101D9000C3EF13FFEE13FEB1CDB1C9C3EA13308711
:101DA000024480FA30E703632201C3E52313F523DD
:101DB000E52213F52250066323A0632201D526D91C
:101DC000E52265236523F52222AE24AF250E0FDE22
:101DD000FEDFFCD20122424C48656C693437316326
:041DE000F390060175
:00000001FF
